:020000040000FA
:04000000CF303A289B
:040004000034003490
:08000800A000030EA100831209
:100010008B1C32288B1032181428B21C3228643002
:10002000010203183128182800001628172818285C
:1000300019281A281B281C281D281E281F283210A2
:10004000B214A810031005190314AA0DA90DA80DC8
:10005000B10B322832152A08AF002908AE00280853
:10006000AD00B21081010B11210E8300A00E200EF5
:02007000090085
:0C007400203084008001840A80300402E7
:10008000031C3C281230B100FF2183160C3085057B
:1000900087018312850187010730990000309A009B
:1000A000103083168E008312603083168F00831207
:1000B00000308316910000008312C830831681003F
:1000C000831231309000003083168C008312103080
:1000D0008B00BD1B7128851971286400851D6D2852
:1000E00037231A2381018E018F010B118B100B1006
:1000F0008C018B17892032199F20B40B872803109D
:1001000085190314BA0DF0303A02031957217D23E3
:100110007A286400321808000B1D08000B11B21079
:1001200032141230B100051D9A28331483160113BE
:10013000831208003310831601178312080032114E
:100140000130B7008B132030370783169B001C1437
:100150001A088312A400A500C030A5061030370786
:1001600083169B001C141A088312A3000030370763
:1001700083169B001C141A088312A2008B17331CD1
:10018000C72822090339A200A309A409A509220846
:100190002D02031D512923082E02031D5129240875
:1001A0002F02031D512901303702031DDC283E18A0
:1001B000DC283E143F14212202303702031DE528BB
:1001C000BE18E528BE143F14302203303702031D49
:1001D000EE283E19EE283E153F143C22043037022B
:1001E000031DF728BE19F728BE153F144822053015
:1001F0003702031D00293E1A00293E163F145722DC
:1002000006303702031D0929BE1A0929BE163F14FC
:10021000662207303702031D12293E1B12293E17A2
:100220003F14752208303702031D1B29BE1B1B29F2
:10023000BE173F14842209303702031D24295E189B
:1002400024295E143F148F220A303702031D2D2902
:10025000DE182D29DE143F149A220B303702031DBD
:1002600036295E1936295E153F14A5220C30370257
:10027000031D3F29DE193F29DE153F14B0220D3042
:100280003702031D48295E1A48295E163F14BB2217
:100290000E303702031D5129DE1A5129DE163F1494
:1002A000C622B70A0F30370203180800A22801300F
:1002B000B600B400B500B70085018701B21317235B
:1002C0008920B40B7029031085190314BA0DF0307E
:1002D0003A0203199729B50B70299630B500A3216E
:1002E000321D60293211331C7A292D090339AD00E2
:1002F000AE09AF092F1CB2132F1C6029B21B602955
:100300002E186029B2178B1320303707BC002F0836
:10031000BB00EA2110303707BC002E08BB00EA21E1
:1003200000303707BC002D08BB00EA218B17850180
:100330008701B70AB6010130B5000F303702031C40
:1003400060291A230800013037020319D122023034
:1003500037020319D622033037020319DB22043097
:1003600037020319E022053037020319E52206306F
:1003700037020319EA22073037020319EF22083047
:1003800037020319F422093037020319F9220A301F
:1003900037020319FE220B303702031903230C30F6
:1003A0003702031908230D30370203190D230E30CD
:1003B00037020319122308003F1C08003F101030B9
:1003C000BC003E08BB00EA213030BC005E08BB0028
:1003D000EA2108008B133B0883161C159A00831230
:1003E0003C0883169B0055309D00AA309D009C144C
:1003F00064009C18F8291C1183128B1708008316BF
:1004000000309B001C141A088312BD0083161030A4
:100410009B001C141A088312BE00831630309B0008
:100420001C141A088312DE00FF30C800CA15CB1551
:10043000CC15CD15CE15CF15D015D115D215D31598
:1004400008008130BE05FF30DE050130C405C00064
:100450000030C200C600BD185F14BD18DF140800CC
:100460008230BE05FF30DE050230C405C00000301A
:10047000C200C6005F1008008430BE05FF30DE05F4
:100480000630C405C0000030C200C6005F1008007E
:100490008830BE05FF30DE050930C405C0000830D5
:1004A000C200C600BD185F14BD18DF1408009030EC
:1004B000BE05FF30DE051930C405C0000030C200A3
:1004C000C600BD185F14BD18DF140800A030BE05BB
:1004D000FF30DE052130C405C0000030C200C60078
:1004E000BD185F14BD18DF140800C030BE05FF3012
:1004F000DE051030C405C0000030C200C600BD18C3
:100500005F14BD18DF140800FF30BE05C030DE05E3
:100510005030C505C1000030C300C70008007F305F
:10052000BE05C130DE052030C505C1000030C30066
:10053000C70008007F30BE05C230DE05E030C505CB
:10054000C1002030C300C70008007F30BE05C430A2
:10055000DE055030C505C1000030C300C7000800EB
:100560007F30BE05C830DE055030C505C100003003
:10057000C300C70008007F30BE05D030DE05503014
:10058000C505C1000030C300C70008007F30BE05AC
:10059000E030DE054030C505C1000030C300C700B3
:1005A00008001030850600308706080020308506D8
:1005B00000308706080021308506003087060800D5
:1005C000123085060030870608001230850602309A
:1005D00087060800103085060430870608000030C2
:1005E0008506023087060800003085061130870630
:1005F0000800003085062030870608000030850698
:10060000383087060800003085061130870608005C
:10061000003085061130870608000030850611304D
:1006200087060800003085063930870608003E1826
:10063000D12208003E182122BE1830223E193C2249
:10064000BE1948223E1A5722BE1A66223E1B752248
:10065000BE1B84225E188F22DE189A225E19A52204
:10066000DE19B0225E1ABB22DE1AC6220800B601CD
:10067000B401B5013D1C3F2BBD01BD14412BBD0193
:100680003D143D08B6006400452B462B472B482BF4
:10069000492BFF30B51B8500B51F8501B40B432BDB
:1006A000B50B432B0310B60CB608031D432B0030CB
:1006B000BC003D08BB00EA21080005125C180516C5
:1006C000DC1C8512DC1885165C1D05105C190514F0
:1006D000DC1D8510DC1985145C1E87105C1A8714DC
:1006E000DC1E0711DC1A07155C1F07105C1B0714C2
:1006F000DC1F8712DC1B871608008F08031908000F
:100700008F0178308E00C80FAF2DC80A441CAD2B66
:10071000461C9E2BCA1C8F2BCA014A15BB2B4A1D97
:10072000942BCA01CA15BB2BCA1D992BCA014A16A4
:10073000BB2B4A1EBB2BCA01CA14BB2B4A1DA32BC1
:10074000CA014A16BB2BCA1DA82BCA014A16BB2BCD
:100750004A1EBB2BCA01CA14BB2BCA1CB22BCA012E
:100760004A15BB2B4A1DB72BCA01CA15BB2B4A1E03
:10077000BB2BCA014A15C41CE22BC61CD32BCB1CB5
:10078000C42BCB014B15F02B4B1DC92BCB01CB152B
:10079000F02BCB1DCE2BCB014B16F02B4B1EF02B91
:1007A000CB01CB14F02B4B1DD82BCB014B16F02BD0
:1007B000CB1DDD2BCB014B16F02B4B1EF02BCB01B1
:1007C000CB14F02BCB1CE72BCB014B15F02B4B1D87
:1007D000EC2BCB01CB15F02B4B1EF02BCB014B158B
:1007E000441D172C461D082CCC1CF92BCC014C1594
:1007F000252C4C1DFE2BCC01CC15252CCC1D032CFF
:10080000CC014C16252C4C1E252CCC01CC14252CAF
:100810004C1D0D2CCC014C16252CCC1D122CCC01C2
:100820004C16252C4C1E252CCC01CC14252CCC1C74
:100830001C2CCC014C15252C4C1D212CCC01CC158D
:10084000252C4C1E252CCC014C15C41D4D2CC61D31
:100850003E2CCD1C2F2CCD014D155F135B2C4D1D57
:10086000342CCD01CD155B2CCD1D392CCD014D1671
:100870005B2C4D1E5B2CCD01CD145B2C4D1D432CF0
:10088000CD014D165B2CCD1D482CCD014D165B2C9A
:100890004D1E5B2CCD01CD145B2CCD1C522CCD01FB
:1008A0004D155B2C4D1D572CCD01CD155B2C4D1ED0
:1008B0005B2CCD014D155F1B842C441E842C461EE1
:1008C000752CCE1C662CCE014E15922C4E1D6B2C19
:1008D000CE01CE15922CCE1D702CCE014E16922C30
:1008E0004E1E922CCE01CE14922C4E1D7A2CCE018F
:1008F0004E16922CCE1D7F2CCE014E16922C4E1EE3
:10090000922CCE01CE14922CCE1C892CCE014E15E9
:10091000922C4E1D8E2CCE01CE15922C4E1E922C5A
:10092000CE014E15C41EB92CC61EAA2CCF1C9B2C62
:10093000CF014F15C72C4F1DA02CCF01CF15C72CB1
:10094000CF1DA52CCF014F16C72C4F1EC72CCF0192
:10095000CF14C72C4F1DAF2CCF014F16C72CCF1D66
:10096000B42CCF014F16C72C4F1EC72CCF01CF146C
:10097000C72CCF1CBE2CCF014F15C72C4F1DC32C2D
:10098000CF01CF15C72C4F1EC72CCF014F15DF1835
:10099000F02C451EF02C471EE12CD01CD22CD0018F
:1009A0005015FE2C501DD72CD001D015FE2CD01D7B
:1009B000DC2CD0015016FE2C501EFE2CD001D01481
:1009C000FE2C501DE62CD0015016FE2CD01DEB2C19
:1009D000D0015016FE2C501EFE2CD001D014FE2C3F
:1009E000D01CF52CD0015015FE2C501DFA2CD00136
:1009F000D015FE2C501EFE2CD0015015DF18272DCF
:100A0000C51E272DC71E182DD11C092DD10151152A
:100A1000352D511D0E2DD101D115352DD11D132D83
:100A2000D1015116352D511E352DD101D114352D41
:100A3000511D1D2DD1015116352DD11D222DD10154
:100A40005116352D511E352DD101D114352DD11C06
:100A50002C2DD1015115352D511D312DD101D1151F
:100A6000352D511E352DD1015115DF185F2D451F34
:100A70005F2D471F502DD21C412DD2015215DF137F
:100A80006D2D521D462DD201D2156D2DD21D4B2D2F
:100A9000D20152166D2D521E6D2DD201D2146D2D24
:100AA000521D552DD20152166D2DD21D5A2DD20137
:100AB00052166D2D521E6D2DD201D2146D2DD21CE9
:100AC000642DD20152156D2D521D692DD201D21502
:100AD0006D2D521E6D2DD2015215DF18982DDF1B82
:100AE000982DC51F982DC71F892DD31C7A2DD30192
:100AF0005315A62D531D7F2DD301D315A62DD31D20
:100B0000842DD3015316A62D531EA62DD301D31425
:100B1000A62D531D8E2DD3015316A62DD31D932D17
:100B2000D3015316A62D531EA62DD301D314A62DE3
:100B3000D31C9D2DD3015315A62D531DA22DD301DA
:100B4000D315A62D531EA62DD3015315DC21400825
:100B5000C4004108C5005F18DF145F1CDF1048089F
:100B6000C9000C304A05031D05120C304B05031D4E
:100B700085120C304C05031D05100C304D05031D6E
:100B800085100C304E05031D87100C304F05031DDA
:100B900007110C305005031D07100C305105031DC3
:100BA00087120C305205031D07120C305305031D2C
:100BB000871149080E020318092E12304A05031D39
:100BC000051612304B05031D851612304C05031D0A
:100BD000051412304D05031D851412304E05031DFA
:100BE000871412304F05031D071512305005031DE1
:100BF000071412305105031D871612305205031DCC
:100C0000071612305305031D8715FF3048020319DC
:100C100008008F08031D0800892049080E02031CE4
:100C2000092E18304A05031D051206304A05031D1A
:100C3000051618304B05031D851206304B05031DA4
:100C4000851618304C05031D051006304C05031D94
:100C5000051418304D05031D851006304D05031D84
:100C6000851418304E05031D871006304E05031DF0
:100C7000871418304F05031D071106304F05031D5B
:100C8000071518305005031D071006305005031DC9
:100C9000071418305105031D871206305105031D36
:100CA000871618305205031D071206305205031D22
:100CB000071618305305031D871106305305031D11
:040CC000871508008C
:084000000700030007000100A6
:02400E00CC33B1
:10420000010003000300030003000200020002009B
:104210000200000000000000000003000300030093
:10422000810000000000000000000000000000000D
:104230000000C000C000C000C000C000C000C0003E
:10424000FF00C300F300CF00FF00C300F300CF0066
:10425000FF00C300F300CF00FF00C300F300CF0056
:104260000000FF00FF00FF00FF00FF00FF00FF0055
:10427000FF00FF00FF00FF00FF00FF00FF00FF0046
:10428000FF000300FF00FF00FF00FF00FF00FF0032
:10429000FF00FF00FF00FF00FF00FF00FF00FF0026
:1042A000FF00C000FF00FF00FF00FF00FF00FF0055
:1042B000FF00FF00FF00FF00FF00FF00FF00FF0006
:1042C000FF00FF00FF00FF00FF00FF00FF00FF00F6
:1042D000FF00FF00FF00FF00FF00FF00FF00FF00E6
:1042E000FF00FF00FF00FF00FF00FF00FF00FF00D6
:1042F000FF00FF00FF00FF00FF00FF00FF00AA001B
:00000001FF
